:10800000FEDF07EA000000000000000000000000A2
:108010000000000000000000000000000000000060
:108020000000000000000000000000000000000050
:108030000000000000000000000000000000000040
:108040000000000000000000000000000000000030
:02000004001FDB
:020000040020DA
:1000000002D3A0E3A60000EBFEFFFFEA001080E5AC
:100010001EFF2FE1B010C0E11EFF2FE10010C0E570
:100020001EFF2FE1000090E51EFF2FE10E00A0E172
:100030001EFF2FE110FF2FE11EFF2FE108402DE9E9
:1000400008009FE5F6FFFFEB0840BDE81EFF2FE12B
:100050005450212008402DE91C009FE5F0FFFFEBE4
:10006000010010E3FBFFFF0A10009FE5ECFFFFEB30
:100070000840BDE8FF0000E21EFF2FE154502120A0
:100080004050212008402DE90C009FE5E4FFFFEBE4
:100090000840BDE8010000E21EFF2FE1545021207E
:1000A00010402DE90040A0E11C009FE5DCFFFFEBC4
:1000B000200010E3FBFFFF0A0410A0E10C009FE505
:1000C000D1FFFFEB1040BDE81EFF2FE1545021206F
:1000D0004050212008402DE910009FE5D0FFFFEBA4
:1000E000010C10E3FBFFFF1A0840BDE81EFF2FE1E3
:1000F0005450212038402DE90050A0E12040A0E3D9
:10010000044044E23534A0E10F3003E2090053E338
:100110003700838230008392E0FFFFEB000054E35E
:10012000F6FFFF1A2000A0E33840BDE8DBFFFFEA3E
:1001300008402DE9EEFFFFEB0D00A0E3D7FFFFEB3A
:100140000A00A0E30840BDE8D4FFFFEA10402DE913
:10015000D8009FE50110A0E3ABFFFFEBD0009FE5C7
:100160000010A0E3A8FFFFEBC8009FE50010A0E38C
:10017000A5FFFFEBC0009FE50310A0E3A2FFFFEB8C
:10018000B8009FE50010A0E39FFFFFEBA0009FE5F4
:100190000010A0E39CFFFFEBA4009FE5C610A0E3C6
:1001A00099FFFFEB9C109FE59C009FE596FFFFEBFE
:1001B00098009FE59AFFFFEB3F1AC0E3121A81E314
:1001C00088009FE590FFFFEB84009FE50010A0E30F
:1001D0008DFFFFEB0040A0E30400A0E1014084E2BA
:1001E00094FFFFEB960054E3FAFFFF1A64009FE5CB
:1001F0000319A0E384FFFFEB0040A0E30400A0E1AB
:10020000014084E28BFFFFEB960054E3FAFFFF1AF4
:1002100040009FE50010A0E37BFFFFEB14009FE58B
:100220000310A0E378FFFFEB1040BDE81EFF2FE1B5
:100230000450212044502120605021204C50212086
:1002400050502120485021200E01000068502120EC
:1002500004002020940020209800202010402DE948
:100260001C409FE5F918A0E30400A0E166FFFFEB46
:100270000400A0E10C109FE563FFFFEB1040BDE818
:100280001EFF2FE108B400200002F90008402DE90C
:1002900008009FE562FFFFEB0840BDE81EFF2FE16D
:1002A00020B40020F8432DE9A7FFFFEB44029FE5AF
:1002B0009EFFFFEB5CFFFFEB9CFFFFEB4900A0E321
:1002C00076FFFFEB4800A0E374FFFFEB4500A0E3DF
:1002D00072FFFFEB5800A0E370FFFFEB0D00A0E3FF
:1002E0006EFFFFEB0A00A0E36CFFFFEB0070A0E3E2
:1002F0000780A0E10760A0E10750A0E10790A0E11E
:100300000740A0E152FFFFEB3A0050E32A00000A49
:100310000D0050E35400000A0A0050E35200000AA6
:100320002030C0E3470053E35100000A013044E2AB
:10033000140053E303F19F97F1FFFFEAAC032000A1
:10034000AC0320004804200048042000480420009A
:100350004804200028042000F4032000D0032000DB
:10036000D0032000D0032000D0032000C4032000CD
:1003700090032000900320009003200090032000B1
:1003800090032000900320009003200090032000A1
:10039000390050E3070040820882A0E10F0000E22C
:1003A000150054E3088080E14200000A28FFFFEBBB
:1003B0003A0050E3014084E2D4FFFF1A0140A0E379
:1003C000CFFFFFEA0662A0E10040A0E3CCFFFFEA16
:1003D000390050E3070040820662A0E10F0000E20E
:1003E000066080E10668A0E12668A0E1014084E2A1
:1003F000C3FFFFEA390050E3070040820552A0E145
:100400000F0000E2055080E1FF5005E2010055E3D6
:100410003400000A3100003A020055E30940A0030D
:100420000040A013B6FFFFEA390050E30700408206
:100430000552A0E10F0000E2055080E1FF5005E207
:100440000840A0E3AEFFFFEA390050E30700408216
:100450000992A0E10F0000E2099080E10998A0E173
:10046000299886E1014084E2A5FFFFEA0040A0E36D
:10047000A3FFFFEA0D00A0E308FFFFEB2D00A0E3C0
:1004800006FFFFEB2D00A0E304FFFFEB0D00A0E350
:1004900002FFFFEB0A00A0E300FFFFEB0A00A0E36E
:1004A000FEFEFFEB0209A0E3E1FEFFEB0000A0E38C
:1004B000F843BDE81EFF2FE1683828E02334A0E1AF
:1004C000FF3CC3E3688423E00900A0E10810A0E139
:1004D000CDFEFFEB097087E0087087E0049089E2A9
:1004E0000E40A0E386FFFFEA0700A0E10FFFFFEB4D
:0C04F0000040A0E382FFFFEA78563412BF
:040000030000800079
:00000001FF
